:0A00000012C0FECFFDCFFCCFFBCFF6
:10000A00FACFF9CFF8CFF7CF26C0F5CFF4CFF3CF99
:10001A00F2CFF1CFF0CFEFCFEECFEDCFF894EE27BE
:10002A00ECBBF1E0FBBFEBBFE5BFF8E1F1BDE1BD21
:10003A008DE0A2E0BB27ED938A95E9F780E094E092
:10004A00A0E6ED930197E9F7EFE5EDBFE4E0EEBF37
:10005A00C0E6D1E098C0AA93EA93EFB7EA9362D5D3
:10006A00AF5FA0936001A150A43A20F05ED5E0E012
:10007A00E0936001E091610155D5EA1708F45AD579
:10008A00E09162014FD5EA1708F457D5E091630170
:10009A0049D5EA1708F454D5E991EFBFE991A99136
:1000AA00189551D5153A28F453D555D557D51F5F0C
:1000BA00F9CF10E0153A28F4109361014FD51F5F6C
:1000CA00F9CF5EC040D5153A30F450D541D550D558
:1000DA0052D51F5FF8CF10E0153A30F447D5109388
:1000EA00620149D51F5FF8CF4BC02DD5153A38F4B8
:1000FA003DD5E4EA3DD52CD544D51F5FF7CF10E0B6
:10010A00153A30F433D5E4EA33D540D51F5FF8CF3A
:10011A0037C019D5153A40F41BD51DD519D528D5A0
:10012A0017D52FD51F5FF6CF10E0153A38F4109384
:10013A006101109362012AD51F5FF7CF21C003D551
:10014A00153A30F41093610103D51BD51F5FF8CF20
:10015A0010E0153A48F410936301FAD409D5A9813D
:10016A00BA8184D61F5FF5CF10E0153A48F4109390
:10017A006201EED4F0D4A981BA8178D61F5FF5CF97
:10018A00188123960895EFEFE7BBE4BBE1BBCDD41A
:10019A00E1E0E9BFE3BF7894A5E0B0E082DFA5E043
:1001AA00B0E090DFA5E0B0E0A0DFAAE0B0E0B1DF08
:1001BA00AAE5B0E0C4DFF894C098B7D4C19AEBD4EA
:1001CA00C198C29AE8D4C298C39AE5D4C398C49A8B
:1001DA00E2D4C498C59ADFD4C598C69ADCD4C69826
:1001EA00C79AD9D4C798A89AD6D4A898A99AD3D482
:1001FA00A998AA9AD0D4AA98AB9ACDD4AB98AC9A1B
:10020A00CAD4AC98AD9AC7D4AD98909AC4D49098F1
:10021A00919AC1D49198929ABED49298939ABBD447
:10022A009398949AB8D49498959AB5D49598969A9E
:10023A00B2D49698979AB2D47DD47FD481D4B1D4CB
:10024A0074D4AFD477D479D47BD4ABD46ED4A9D4B4
:10025A0071D473D475D4A5D468D4A3D46BD46DD413
:10026A006FD49FD462D49DD465D467D469D499D409
:10027A005CD497D45FD461D463D4A0E9B1E0F6D555
:10028A0054D4AAEF91D459D491D495D48FD495D477
:10029A008DD495D48BD495D489D495D487D495D438
:1002AA0085D491D483D48BD481D487D47FD487D472
:1002BA007DD487D47BD47FD479D47FD477D485D4A2
:1002CA0075D479D473D479D471D479D46FD479D4D8
:1002DA006DD479D46BD479D469D475D467D46FD4F6
:1002EA0065D46BD463D46BD461D46BD45FD463D438
:1002FA005DD463D45BD469D459D465D457D45FD45C
:10030A0055D45FD453D45FD451D45FD44FD4E5BB12
:10031A00EFE7E8BB4BD453D449D44FD447D44FD496
:10032A0045D44FD443D447D441D447D43FD44DD4F1
:10033A003DD441D43BD441D439D441D437D441D427
:10034A0035D441D433D441D431D43DD42FD437D445
:10035A002DD433D42BD433D429D433D427D42BD487
:10036A0025D42BD423D431D421D4E2BBE0E0E5BB9D
:10037A00E8BB17D4C19AC29A2AD4C3982BD4C59A77
:10038A00C69A25D4C79828D4A99AAA9A20D4AB98F1
:10039A0025D4AD9A909A1BD4919822D4939A949A80
:1003AA0016D495981FD420D4C39AC49A21D4C79A34
:1003BA00A89A1ED4AB9AAC9A1BD4919A929A18D442
:1003CA00959A969A15D410D4B0D3EBD3979AC19A2A
:1003DA0012D4969AC29A0FD4959AC39A0CD4949A24
:1003EA00C49A09D4C59A939A06D4C69A929A03D4FF
:1003FA00C79A919A00D4909AA89AFDD3A99AAD9ACD
:10040A00FAD3FCD3F8D3AB9ACCD38FD3FAD3FCD399
:10041A00FDD3FAD3FDD3FAD3F7D3FAD3FBD3FCD364
:10042A00F5D3F2D3F5D3F6D3F9D3FAD3F5D3EED382
:10043A00EBD3EED3EFD3F2D3F5D3F6D3F1D3ECD398
:10044A00E5D3E2D3E5D3E6D3E9D3ECD3EFD3F0D3C4
:10045A00EBD3E6D3E1D3DAD3D7D3DAD3DBD3DED304
:10046A00E1D3E4D3E7D3E8D3E3D3DED3D9D3D4D3E8
:10047A00CDD3CAD3CDD3CED3D1D3D4D3D7D3DAD352
:10048A00DDD3DED3D9D3D4D3CFD3CAD3C5D3BED346
:10049A00BBD3BED3BFD3C2D3C5D3C8D3CBD3CED39A
:1004AA00D1D3D2D3CDD3C8D3C3D3BED3B9D3B4D384
:1004BA00ADD3AAD3ADD3AED3B1D3B4D3B7D3BAD312
:1004CA00BDD3C0D3C3D3C4D3BFD3BAD3B5D3B0D3A8
:1004DA00ABD3A6D3A1D39AD397D39AD39BD39ED384
:1004EA00A1D3A4D3A7D3AAD3ADD3B0D3B3D3B4D310
:1004FA00AFD3AAD3A5D3A0D39BD396D391D38CD36E
:10050A0085D386D387D38AD38DD390D393D396D3E7
:10051A0099D39CD39FD3A2D3A3D39ED399D394D355
:10052A008FD38AD385D380D37BD376D36FD36CD33F
:10053A006FD370D373D376D379D37CD37FD382D35B
:10054A0085D388D38BD38ED38FD38AD385D380D3C5
:10055A007BD376D371D36CD367D362D35DD356D3AF
:10056A0053D356D357D35AD35DD360D363D366D309
:10057A0069D36CD36FD372D375D378D379D374D349
:10058A006FD36AD365D360D35BD356D351D34CD3DD
:10059A0047D342D33BD338D33BD33CD33FD342D3C5
:1005AA0045D348D34BD34ED351D354D357D35AD32D
:1005BA005DD360D361D35CD357D352D34DD348D3E1
:1005CA0043D33ED339D334D32FD32AD325D31ED3FF
:1005DA001BD31ED31FD322D325D328D32BD32ED359
:1005EA0031D334D337D33AD33DD340D343D346D38D
:1005FA0047D342D33DD338D333D32ED329D324D3AD
:10060A001FD31AD315D310D30BD306D3FFD2FCD2E0
:10061A00FFD200D303D306D309D30CD30FD312D3FB
:10062A0015D318D31BD31ED321D324D327D32AD32C
:10063A002BD326D321D31CD317D312D30DD308D34C
:10064A0003D3FED2F9D2F4D2EFD2EAD2E5D2DED285
:10065A00DBD2DED2DFD2E2D2E5D2E8D2EBD2EED2E0
:10066A00F1D2F4D2F7D2FAD2FDD200D303D306D311
:10067A0009D30CD3C598C5D207D302D3FDD2F8D279
:10068A00F3D2EED2E9D2E4D2DFD2DAD2D5D2D0D2C4
:10069A00CBD2C6D2C1D2BAD2B7D2BAD2BBD2BED2CA
:1006AA00C1D2C4D2C7D2CAD2CDD2D0D2D3D2D6D254
:1006BA00D9D2DCD2DFD2E2D2E5D2E8D2C39AA1D231
:1006CA00C4989FD2C5989DD2DFD2DAD2D5D2D0D2E1
:1006DA00CBD2C6D2C1D2BCD2B7D2B2D2ADD2A8D2B4
:1006EA00A3D29ED299D292D28FD292D293D296D2BA
:1006FA0099D29CD29FD2A2D2A5D2A8D2ABD2AED244
:10070A00B1D2B4D2B7D2BAD2BDD2C0D2C39A79D2F8
:10071A00C29A77D2C39875D2C49873D2C59871D247
:10072A00B3D2AED2A9D2A4D29FD29AD295D290D223
:10073A008BD286D281D27CD277D272D26DD266D255
:10074A0063D266D267D26AD26DD270D273D276D2AF
:10075A0079D27CD27FD282D285D288D28BD28ED2E3
:10076A0091D294D2C39A4DD2C29A4BD2C19A19D27B
:10077A00C19817D2C29815D2C39813D2C49811D26D
:10078A00C5980FD2C6980DD2C7980BD2A89809D28D
:10079A00A99807D2AA9805D2AB9803D2AC9801D2ED
:1007AA00AD98FFD19098FDD19198FBD19298F9D14B
:1007BA009398F7D19498F5D19598F3D19698F1D169
:1007CA009798EFD165D264D266D269D26CD26FD2D1
:1007DA0072D275D278D27BD27ED281D284D287D29B
:1007EA008AD28DD290D293D296D299D29CD29FD2CB
:1007FA00A2D2A5D2A8D295984BD2A9D2ACD2AFD2C6
:10080A00B2D2C29845D247D24AD24DD250D253D24E
:10081A0056D259D25CD25FD262D265D268D26BD23A
:10082A006ED271D274D277D27AD27DD280D283D26A
:10083A0086D289D295982CD28AD28DD290D293D24E
:10084A00C29826D228D22BD22ED231D234D237D243
:10085A003AD23DD240D243D246D249D24CD24FD2DA
:10086A0052D255D258D25BD25ED261D264D267D20A
:10087A006AD295980DD26BD26ED257D192D1C09AC4
:10088A0076D277D279D27BD27CD27ED280D282D2F1
:10089A0083D285D287D289D28AD28CD28ED290D272
:1008AA0091D293D295D2959A9DD1969A94D25FD2AB
:1008BA0060D262D264D265D267D269D26BD26CD26C
:1008CA006ED270D272D273D275D277D279D27AD2EC
:1008DA007CD27ED2959A86D14AD24BD24DD24FD271
:1008EA0050D252D254D256D257D259D25BD25DD2BA
:1008FA005ED260D262D264D265D267D269D237D26E
:10090A0038D23AD23CD23DD23FD241D243D244D25B
:10091A0046D248D24AD24BD24DD24FD251D252D2DB
:10092A0054D225D226D228D22AD22BD22DD22FD2B5
:10093A0031D232D234D236D238D239D23BD23DD267
:10094A003FD240D214D215D217D219D21AD21CD2FF
:10095A001ED220D221D223D225D227D228D22AD2DD
:10096A002CD22ED204D205D207D209D20AD20CD264
:10097A000ED210D211D213D215D217D218D21AD23D
:10098A001CD2F5D1F6D1F8D1FAD1FBD1FDD1FFD1E4
:10099A0001D202D204D206D208D209D20BD2E7D1AE
:1009AA00E8D1EAD1ECD1EDD1EFD1F1D1F3D1F4D143
:1009BA00F6D1F8D1FAD1FBD1DAD1DBD1DDD1DFD151
:1009CA00E0D1E2D1E4D1E6D1E7D1E9D1EBD1EDD161
:1009DA00CED1CFD1D1D1D3D1D4D1D6D1D8D1DAD1E8
:1009EA00DBD1DDD1DFD1C3D1C4D1C6D1C8D1C9D100
:1009FA00CBD1CDD1CFD1D0D1D2D1D1D1B8D1B9D11A
:100A0A00BBD1BDD1BED1C0D1C2D1C4D1A998DFD08A
:100A1A00AED1AFD1B1D1B3D1B4D1B6D1B8D1A7D1BA
:100A2A00A8D1AAD1ACD1ADD1AFD1A1D1A2D1A4D1F3
:100A3A00A6D1A7D1C19ACBD09CD19ED1A0D197D112
:100A4A0098D19AD194D195D192D1E0E8E8BBE0E06F
:100A5A00E5BBE2BBA3D0C09AC0D1C9D1CDD1DAD10E
:100A6A00C6D1CAD1D7D1C3D1C7D1DFD1E1D1969AE4
:100A7A00B4D1BDD1C1D1CED1BAD1BED1CBD1B7D1EA
:100A8A00BBD1C8D1B4D1B8D1DBD1949AA6D1AFD158
:100A9A00B3D1C0D1ACD1B0D1D3D1969AC6D1D3D12A
:100AAA009398959898D1D6D1CED194989BD0B2D11B
:100ABA009ED1909A929A959AA8E7B5E0D7D18DD10E
:100ACA0096D19AD1A7D193D197D1A4D190D194D1CB
:100ADA00ACD1AED1969A81D18AD18ED19BD187D110
:100AEA008BD198D184D188D195D181D185D1A8D102
:100AFA00949A73D17CD180D18DD179D17DD1A0D175
:100B0A00969A93D1A0D19398959865D1A3D19BD168
:100B1A00949868D07FD16BD1909A929A959A3ED048
:100B2A003ACBFFCFA09160010895E0E0E8BBE5BBB6
:100B3A00E2BB0895EEEFE8BB0895EFE3E5BB089545
:100B4A00EFEFE2BB0895BA93AA931A9310E00895BF
:100B5A00E4EAE11B0895E09361010895E4EAE09371
:100B6A006201E0936301A981BA8180C1E4EAF3CF0B
:100B7A00E09362010895E4EAE0936301A981BA81EE
:100B8A0075C1E0936301A981BA8170C110936301B1
:100B9A00A981BA816BC1A4E1B5E068C1A8EEB3E04E
:100BAA0065C1ACE2B1E062C1B0E060C1A4EFB1E0FE
:100BBA005DD1E0E00895E5BBC3CFE2BBBBCFE8BBA4
:100BCA00BFCFE2BBBACFE5BBB5CFE8BBB6CFA4EA8D
:100BDA00B6E04CC1C498FBCFA898F9CFAC98F7CF30
:100BEA009298F5CF9698F3CF979AACEABDE03EC1BA
:100BFA00ACEABDE03BC1ACEFB8E038C1AA9AAC9A06
:100C0A000895A4EFB1E032C1979AFBCF9798F9CF34
:100C1A00969AF7CF959AF5CF9698F3CF949AF1CF03
:100C2A009598EFCF939AEDCF9498EBCF929AE9CF1C
:100C3A009398E7CF919AE5CF9298E3CF909AE1CF34
:100C4A009198DFCFAD9ADDCF9098DBCFAC9AD9CF10
:100C5A00AD98D7CFAB9AD5CFAC98D3CFAA9AD1CFEC
:100C6A00AB98CFCFA99ACDCFAA98CBCFA89AC9CF04
:100C7A00A998C7CFC79AC5CFA898C3CFC69AC1CFDC
:100C8A00C798BFCFC59ABDCFC698BBCFC49AB9CFB4
:100C9A00C79AA8EC89CFC798AD9AA8EC85CFAD982A
:100CAA00979AA8EC81CF9798C19AA8EC7DCFC19862
:100CBA00919AA8EC79CF9198A99AA8EC75CFA9989E
:100CCA00969AA8EC71CF9698C39AA8EC6DCFC39860
:100CDA00939AA8EC69CF9398AA9AA8EC65CFAA9898
:100CEA00949AA8EC61CF9498C59AA8EC5DCFC59860
:100CFA00909AA8EC59CF9098C49AA8EC55CFC4986A
:100D0A00AC9AA8EC51CFAC98929AA8EC4DCF929895
:100D1A00C19AA8EC49CFC198979AA8EC45CF979861
:100D2A00C69AA8EC41CFC698AB9AA8EC3DCFAB982F
:100D3A00949AA8EC39CF9498A89AA8EC35CFA89899
:100D4A00C19AA8EC31CFC198959AA8EC2DCFC79833
:100D5A00939AA8EC29CF9398C49AA8EC25CFC49863
:100D6A00AD9AA8EC21CFAD98C29AA8EC1DCFC19834
:100D7A002ECFC19AC2982BCFC29AC39828CFC39AB2
:100D8A0029CFC49AC59823CFC59AC69820CFC69AA8
:100D9A00C7981DCFC79A20CFA89AA99818CFA99A01
:100DAA00AA9815CFAA9AAB9812CFAB9A17CFAC9A3A
:100DBA00AD980DCFAD9A90980ACF909A919807CF97
:100DCA00919A0ECF929A939802CF939A9498FFCEC3
:100DDA00949A9598FCCE9798FACEC298C498C698D9
:100DEA00A898AA98AC98909892989598F4CFC29A95
:100DFA00C49AC69AA89A02CF909A929A959A979A62
:100E0A00C198C398C598C798A998AB98AD98919876
:100E1A009498E8CEC19AC39AC59AC79AA99AAB9AE6
:100E2A00AD9A919A949A969AD8CFC198C3980895F0
:100E3A00C59AC79AA99AAB9AAD9A919A949A089523
:100E4A00C19AC39AF5CFC598C798A998AB98AD9897
:100E5A0091980895C19AC39AC59AC79AA99AAB9AC2
:100E6A00AD9A919A939A959A979ADFCF109639F0FC
:100E7A0088EC90E00197F1F7A8951197C9F70895C2
:00000001FF
